:10000000D529A701AB01AA000130A5002B082702C2
:10001000031D0C282A082602043003180130031996
:1000200002302505031D0130D1298030A100FE30AA
:10003000F2200130F2207530A70030300629A101EE
:10004000A117B500FE30F2203508F228AE01AF014D
:10005000B001B101A512F520D33E0319A5162D3E1E
:10006000C63E03182B280A3E031C2B28AA00A90110
:10007000A801A7010A30A600AF212A082607AE0072
:100080002708AF00030103180130AF072808B000AC
:10009000030103180130B0072908B1000301031858
:1000A0000130B107A40303195C28F520C63E0318EC
:1000B0005C280A3E03183628A51E6928AE09AF0938
:1000C000B009B109AE0A0319AF0A0319B00A03193E
:1000D000B10A2E08D129A401AE00AF01A011240855
:1000E0000319A0150530A3002730AB001030842081
:1000F0000330AB00E8308420AB0164308420AB01D6
:100100000A3084202E088B28AA002F08A7002E086A
:10011000A60093212608A600A3030319A011240812
:1001200003199528230203189C282608031DA011F3
:10013000A0199C28303EF2280800B3000610861152
:100140008316061086110F30860583123308A01817
:10015000C7283E30A700803006213330B200DB20B4
:100160001330A70088300621DB2064300521DB2016
:10017000643005212230B200DB202830C6200C304C
:10018000C6200630C620A0143308C7282014B200A9
:10019000201CD5288611033C031CDA28DA200730FE
:1001A000A700D0300621031408002014FE3C0319D8
:1001B000E8288615201C201006140F30860532080A
:1001C000F03986040610B20E2018DB28FF30052116
:1001D0003308D1299818181218168C1EED281A0801
:1001E0000314D129A11B9D2808003A030319EA280A
:1001F000AB01AA00FF30AA07031CAB07031CD129DF
:100200000330A700E4300621FA28A701F43EA60037
:10021000A709FE30031C0F29A60703180C29A607FF
:100220000000A70F0C2900002618162926181829E7
:100230000800290831068039B300A91F2A29A60918
:10024000A709A809A909A60A0319A70A0319A80A50
:100250000319A90AB11F3729AE09AF09B009B109BD
:10026000AE0A0319AF0A0319B00A0319B10AAA01A9
:10027000AB01AC01AD01B601B701B801B90131085C
:1002800030042F042E04031975292030B200031006
:10029000A60DA70DA80DA90DB60DB70DB80DB90D7A
:1002A00031083902031D5E2930083802031D5E291A
:1002B0002F083702031D5E292E083602031C6F2902
:1002C0002E08B6022F08031C2F0FB7023008031C9C
:1002D000300FB8023108031C310FB9020314AA0D04
:1002E000AB0DAC0DAD0DB20B4729B31F8229AA0986
:1002F000AB09AC09AD09AA0A0319AB0A0319AC0A88
:100300000319AD0A3608AE003708AF003808B00050
:100310003908B1002A08A6002B08A7002C08A8005D
:100320002D08A900D129AF01AE011030B200270D70
:10033000AE0DAF0D2A08AE022B08031C2B0FAF0227
:100340000318A9292A08AE072B0803182B0FAF079B
:100350000310A60DA70DB20B97292608D12920302E
:10036000B200B601B701B801B9010310261CC629B5
:100370002E08B6072F0803182F0FB70730080318E9
:10038000300FB80731080318310FB907B90CB80C92
:10039000B70CB60CA90CA80CA70CA60CB20BB5296F
:1003A0000800831383120313080083161930990081
:1003B00000309800831290309800A00107309F0011
:1003C000023083168600F130850083127A2A4208B3
:1003D000A9004108A8004008A7003F08A600B101F5
:1003E000B001AF016430AE0019212E08BE004208F2
:1003F000A9004108A8004008A7003F08A600B101D5
:10040000B001AF016430AE0019212908C2002808EC
:10041000C1002708C0002608BF004208A900410803
:10042000A8004008A7003F08A600B101B001AF0135
:100430006430AE0019212E08BD004208A900410811
:10044000A8004008A7003F08A600B101B001AF0115
:100450006430AE0019212608BC000800EA20243CC4
:10046000031D2E2AEA20473C031D2E2AEA20503C79
:10047000031D2E2AEA20523C031D2E2AEA204D3C61
:10048000031D2E2AEA20433C031D2E2AEA202C3C81
:10049000031D2E2A0130BA00A4012620BF002F0818
:1004A000C0003008C1003108C200E721EA20243C26
:1004B000031D562AEA20473C031D562AEA20503CD9
:1004C000031D562AEA20473C031D562AEA20533CC6
:1004D000031D562AEA20413C031D562AEA202C3CE3
:1004E000031D562AEA20C4000130BA00A4012620C8
:1004F000C3000800C301BE01BD01BC010511851187
:10050000851015208030A1001F2047309D205030DD
:100510009D2053309D2020309D2077309D206130DC
:100520009D2069309D2074309D200330AB00E83061
:10053000F9202E220A303C020318A82A8030A1009C
:100540001F2030309D203C086B203A309D20AF2A80
:100550008030A1001F203C086B203A309D200A30DB
:100560003D020318BC2A30309D208030A1003D0898
:100570006B203A309D20C22A8030A1003D086B20BC
:100580003A309D200A303E020318D02A30309D2098
:100590008030A1003E086B2020309D209D20DE2A67
:1005A0008030A1003E086B2020309D2055309D20DA
:1005B00054309D2043309D2020309D200230430246
:1005C000013003180301BB004308A60003300120DB
:1005D000BB040319032B8030A100C0301F204E3014
:1005E0009D206F309D2020309D206C309D206F30ED
:1005F0009D2063309D206B309D2020309D209D20CC
:1006000005158511851002304302031D1F2B803014
:10061000A100C0301F2032309D2044309D2020306A
:100620009D206C309D206F309D2063309D206B306D
:100630009D2020309D209D200511851185140330BB
:100640004302031D3B2B8030A100C0301F203330FC
:100650009D2044309D2020309D206C309D206F30A7
:100660009D2063309D206B309D2020309D209D205B
:0E067000051185158510992A63003C2B3E2B41
:02400E00223F4F
:00000001FF
